:020000040800F2
:10000000000002207D62000827590008CD62000828
:100010002D59000833590008395900080000000024
:100020000000000000000000000000003F59000830
:100030004D590008000000005B590008695900088C
:10004000CD620008CD620008CD620008CD620008D4
:10005000CD620008CD620008CD620008CD620008C4
:10006000CD620008CD620008CD620008CD620008B4
:10007000CD620008CD620008CD620008CD620008A4
:10008000CD620008CD62000879590008CD620008F1
:100090008D590008CD620008A1590008CD62000802
:1000A000B5590008CD620008CD620008CD62000895
:1000B000CD620008CD620008CD620008CD62000864
:1000C000CD620008CD620008CD620008CD62000854
:1000D000CD620008C9590008CD620008CD62000851
:1000E000CD620008CD620008CD620008CD62000834
:1000F000CD620008CD620008CD620008CD62000824
:10010000CD620008CD620008CD620008CD62000813
:10011000CD620008CD620008CD620008CD62000803
:10012000CD620008CD620008E1590008CD620008E8
:10013000CD6200080000000000000000CD62000851
:10014000F5590008CD620008095A0008CD62000880
:10015000CD620008CD6200081D5A0008CD6200087B
:10016000CD620008CD620008CD620008CD620008B3
:10017000CD620008CD620008000000000000000011
:08018000CD620008CD62000809
:1001880010B5054C237833B9044B13B10448AFF3C9
:1001980000800123237010BD4000002000000000F3
:1001A8004463000808B5034B1BB103490348AFF388
:1001B800008008BD000000004400002044630008DF
:1001C80053B94AB9002908BF00281CBF4FF0FF31B6
:1001D8004FF0FF3000F074B9ADF1080C6DE904CEB2
:1001E80000F006F8DDF804E0DDE9022304B070470A
:1001F8002DE9F047089D04468E46002B4DD18A42D2
:10020800944669D9B2FA82F252B101FA02F3C2F104
:10021800200120FA01F10CFA02FC41EA030E944095
:100228004FEA1C48210CBEFBF8F61FFA8CF708FBB6
:1002380016E341EA034306FB07F199420AD91CEB8E
:10024800030306F1FF3080F01F81994240F21C81C0
:10025800023E63445B1AA4B2B3FBF8F008FB103308
:1002680044EA034400FB07F7A7420AD91CEB04043D
:1002780000F1FF3380F00A81A74240F2078164440D
:10028800023840EA0640E41B00261DB1D440002392
:10029800C5E900433146BDE8F0878B4209D9002DF6
:1002A80000F0EF800026C5E9000130463146BDE880
:1002B800F087B3FA83F6002E4AD18B4202D38242EA
:1002C80000F2F980841A61EB030301209E46002D99
:1002D800E0D0C5E9004EDDE702B9FFDEB2FA82F2EE
:1002E800002A40F09280A1EB0C014FEA1C471FFA4C
:1002F8008CFE0126200CB1FBF7F307FB131140EA33
:1003080001410EFB03F0884208D91CEB010103F1FF
:10031800FF3802D2884200F2CB804346091AA4B2C1
:10032800B1FBF7F007FB101144EA01440EFB00FE95
:10033800A64508D91CEB040400F1FF3102D2A645FA
:1003480000F2BB800846A4EB0E0440EA03409CE799
:10035800C6F12007B34022FA07FC4CEA030C20FA46
:1003680007F401FA06F31C43F9404FEA1C4900FA66
:1003780006F3B1FBF9F8200C1FFA8CFE09FB1811E3
:1003880040EA014108FB0EF0884202FA06F20BD956
:100398001CEB010108F1FF3A80F08880884240F2A6
:1003A8008580A8F102086144091AA4B2B1FBF9F0EA
:1003B80009FB101144EA014100FB0EFE8E4508D9E5
:1003C8001CEB010100F1FF346CD28E456AD902386A
:1003D800614440EA0840A0FB0294A1EB0E01A1424F
:1003E800C846A64656D353D05DB1B3EB080261EBBD
:1003F8000E0101FA07F722FA06F3F1401F43C5E997
:10040800007100263146BDE8F087C2F12003D840CC
:100418000CFA02FC21FA03F3914001434FEA1C470E
:100428001FFA8CFEB3FBF7F007FB10360B0C43EA00
:10043800064300FB0EF69E4204FA02F408D91CEBB0
:10044800030300F1FF382FD29E422DD902386344AE
:100458009B1B89B2B3FBF7F607FB163341EA03414E
:1004680006FB0EF38B4208D91CEB010106F1FF389D
:1004780016D28B4214D9023E6144C91A46EA004694
:1004880038E72E46284605E70646E3E61846F8E626
:100498004B45A9D2B9EB020864EB0C0E0138A3E76F
:1004A8004646EAE7204694E74046D1E7D0467BE750
:1004B800023B614432E7304609E76444023842E7C8
:1004C800704700BF80B584B000AF78600023FB732D
:1004D8007B68002B01D1012333E07B681B6C002B68
:1004E80009D1786805F0DAFA7B6800225A647B68DB
:1004F800002283F83C207B681B6C03F01003002B60
:1005080018D17B681B6C23F4885323F0020343F053
:1005180002027B681A64786800F068FA7B68002237
:100528005A647B681B6C23F0030343F001027B6869
:100538001A6401E00123FB737B68002283F83C20E6
:10054800FB7B18461037BD4680BD80B586B000AF2E
:10055800786000237B6100233B617B681B681B6814
:10056800FB607B681B685B68BB60FB6803F0020389
:100578007B61BB6803F020033B617B69002B49D09A
:100588003B69002B46D07B681B6C03F01003002BE3
:1005980005D17B681B6C43F400727B681A647B6826
:1005A8001B689B6803F04053002B2BD17B681B7E94
:1005B800002B27D17B681B68DB6A03F47003002BD0
:1005C80006D07B681B689B6803F48063002B19D1F5
:1005D8007B681B685A687B681B6822F020025A6097
:1005E8007B681B6C23F480727B681A647B681B6CC5
:1005F80003F48053002B05D17B681B6C43F0010288
:100608007B681A64786800F0B0F87B681B686FF044
:1006180012021A60FB6803F004037B61BB6803F0F5
:1006280080033B617B69002B57D03B69002B54D07A
:100638007B681B6C03F01003002B05D17B681B6CD7
:1006480043F400527B681A647B681B689B6803F458
:100658004013002B39D17B681B689B6B03F4401354
:10066800002B06D07B681B689B6803F48063002B13
:100678002BD17B681B685B6803F48063002B24D153
:100688007B681B689B6803F04053002B1DD17B6877
:100698001B7E002B19D17B681B685A687B681B6816
:1006A80022F080025A607B681B6C23F480527B68BE
:1006B8001A647B681B6C03F48073002B05D17B687C
:1006C8001B6C43F001027B681A64786800F08AFAB0
:1006D8007B681B686FF00C021A60FB6803F001036B
:1006E8007B61BB6803F040033B617B69002B17D03B
:1006F8003B69002B14D07B681B681B6803F001035F
:10070800012B0DD17B681B6C43F480327B681A6423
:10071800786800F034F87B681B686FF001021A6093
:10072800FB6803F020037B61BB6803F080633B61D7
:100738007B69002B15D03B69002B12D07B685B6C62
:1007480043F002027B685A647B681B686FF02002E2
:100758001A60786800F01DF87B681B686FF020024B
:100768001A6000BF1837BD4680BD80B483B000AFA3
:10077800786000BF0C37BD465DF8047B704780B4D5
:1007880083B000AF786000BF0C37BD465DF8047BCE
:10079800704780B483B000AF786000BF0C37BD46A7
:1007A8005DF8047B7047000080B485B000AF7860C6
:1007B80039600023BB607B6893F83C30012B01D182
:1007C800022305E17B68012283F83C203B681B6813
:1007D800092B25D97B681B68D9683B681B689BB2C5
:1007E8001A4613465B0013441E3B072202FA03F322
:1007F800DA437B681B680A40DA607B681B68D96843
:100808003B689A683B681B689BB2184603465B00C6
:1008180003441E3B9A407B681B680A43DA6022E067
:100828007B681B6819693B681B689BB21A461346AC
:100838005B001344072202FA03F3DA437B681B6860
:100848000A401A617B681B6819693B689A683B68AB
:100858001B689BB2184603465B0003449A407B68BA
:100868001B680A431A613B685B68062B24D87B68BF
:100878001B68596B3B685A6813469B001344053B39
:100888001F2202FA03F3DA437B681B680A405A63A3
:100898007B681B68596B3B681B689BB218463B68B2
:1008A8005A6813469B001344053B00FA03F27B6821
:1008B8001B680A435A634CE03B685B680C2B24D8DE
:1008C8007B681B68196B3B685A6813469B00134486
:1008D800233B1F2202FA03F3DA437B681B680A40B2
:1008E8001A637B681B68196B3B681B689BB21846C8
:1008F8003B685A6813469B001344233B00FA03F2F3
:100908007B681B680A431A6323E07B681B68D96A03
:100918003B685A6813469B001344413B1F2202FA66
:1009280003F3DA437B681B680A40DA627B681B685A
:10093800D96A3B681B689BB218463B685A681346DD
:100948009B001344413B00FA03F27B681B680A438F
:10095800DA62224BFB607B681B68214A934209D10B
:100968003B681B68122B05D1FB685B6843F4800267
:10097800FB685A607B681B68194A934223D13B681D
:100988001B68102B03D03B681B68112B1BD1FB681D
:100998005B6843F40002FB685A603B681B68102BD5
:1009A80011D1104B1B68104AA2FB03239A0C134663
:1009B8009B0013445B00BB6002E0BB68013BBB606B
:1009C800BB68002BF9D17B68002283F83C20002308
:1009D80018461437BD465DF8047B70470023014074
:1009E800002001403C00002083DE1B4380B485B01A
:1009F80000AF7860794BFB60FB685B6823F440329A
:100A0800FB685A60FB685A687B685B681A43FB6836
:100A18005A607B681B685A687B681B6822F480727E
:100A28005A607B681B6859687B681B691A027B6877
:100A38001B680A435A607B681B685A687B681B6896
:100A480022F040725A607B681B6859687B689A6814
:100A58007B681B680A435A607B681B689A687B68D6
:100A68001B6822F400629A607B681B6899687B683F
:100A7800DA687B681B680A439A607B689B6A584AF5
:100A8800934222D07B681B689A687B681B6822F0B7
:100A980070629A607B681B6899687B689A6A7B6851
:100AA8001B680A439A607B681B689A687B681B68A6
:100AB80022F040529A607B681B6899687B68DA6A02
:100AC8007B681B680A439A600FE07B681B689A681A
:100AD8007B681B6822F070629A607B681B689A6862
:100AE8007B681B6822F040529A607B681B689A6892
:100AF8007B681B6822F002029A607B681B68996811
:100B08007B681B7E5A007B681B680A439A607B6877
:100B180093F82030002B1BD07B681B685A687B68D1
:100B28001B6842F400625A607B681B685A687B68DD
:100B38001B6822F460425A607B681B6859687B68AE
:100B48005B6A013B5A037B681B680A435A6007E0EB
:100B58007B681B685A687B681B6822F400625A60CD
:100B68007B681B68DA6A7B681B6822F47002DA62A9
:100B78007B681B68D96A7B68DB69013B1A057B685F
:100B88001B680A43DA627B681B689A687B681B6883
:100B980022F400729A607B681B6899687B6893F8F6
:100BA80030305A027B681B680A439A607B681B686E
:100BB8009A687B681B6822F480629A607B681B686D
:100BC80099687B685B699A027B681B680A439A602C
:100BD80000BF1437BD465DF8047B70470023014011
:100BE8000100000F80B483B000AF786000BF0C37FD
:100BF800BD465DF8047B704780B586B000AF78606D
:100C08007B68002B01D1012367E27B681B6803F036
:100C18000103002B75D0884B9B6803F00C03042B51
:100C28000CD0854B9B6803F00C03082B12D1824B28
:100C38005B6803F48003B3F5800F0BD17E4B1B6810
:100C480003F40033002B5BD07B685B68002B57D123
:100C5800012342E27B685B68B3F5803F06D1764B9F
:100C68001B68754A43F4803313601DE07B685B683A
:100C7800B3F5A02F0CD1704B1B686F4A43F4802347
:100C880013606D4B1B686C4A43F4803313600BE0B0
:100C9800694B1B68684A23F480331360664B1B68F2
:100CA800654A23F4802313607B685B68002B13D0AC
:100CB80001F062FE386108E001F05EFE02463B6921
:100CC800D31A642B01D9032307E25B4B1B6803F497
:100CD8000033002BF0D014E001F04EFE386108E03C
:100CE80001F04AFE02463B69D31A642B01D903235B
:100CF800F3E1514B1B6803F40033002BF0D100E003
:100D080000BF7B681B6803F00203002B63D04A4BCB
:100D18009B6803F00C03002B0BD0474B9B6803F038
:100D28000C03082B1CD1444B5B6803F48003002B95
:100D380016D1414B1B6803F00203002B05D07B68DA
:100D4800DB68012B01D00123C7E13B4B1B6823F073
:100D5800F8027B681B69DB00374913430B603AE0F4
:100D68007B68DB68002B20D0344B01221A6001F02D
:100D780003FE386108E001F0FFFD02463B69D31A23
:100D8800022B01D90323A8E12B4B1B6803F00203B4
:100D9800002BF0D0284B1B6823F0F8027B681B69F6
:100DA800DB00254913430B6015E0244B00221A6031
:100DB80001F0E2FD386108E001F0DEFD02463B6922
:100DC800D31A022B01D9032387E11B4B1B6803F0BD
:100DD8000203002BF0D17B681B6803F00803002B8B
:100DE80036D07B685B69002B16D0154B01221A6040
:100DF80001F0C2FD386108E001F0BEFD02463B6922
:100E0800D31A022B01D9032367E10B4B5B6F03F065
:100E18000203002BF0D01BE0094B00221A6001F0FE
:100E2800ABFD38610EE001F0A7FD02463B69D31A1D
:100E3800022B07D9032350E1003802400000474243
:100E4800800E4742884B5B6F03F00203002BEAD108
:100E58007B681B6803F00403002B00F097800023D5
:100E6800FB75814B1B6C03F08053002B0FD10023C3
:100E7800BB607D4B1B6C7C4A43F0805313647A4BF8
:100E88001B6C03F08053BB60BB680123FB75774B79
:100E98001B6803F48073002B18D1744B1B68734ACA
:100EA80043F48073136001F067FD386108E001F0D6
:100EB80063FD02463B69D31A022B01D903230CE1D7
:100EC8006A4B1B6803F48073002BF0D07B689B6827
:100ED800012B06D1644B1B6F634A43F00103136770
:100EE8001CE07B689B68052B0CD15F4B1B6F5E4A2F
:100EF80043F0040313675C4B1B6F5B4A43F0010329
:100F080013670BE0584B1B6F574A23F00103136715
:100F1800554B1B6F544A23F0040313677B689B6887
:100F2800002B15D001F028FD38610AE001F024FDFE
:100F380002463B69D31A41F28832934201D903230E
:100F4800CBE0494B1B6F03F00203002BEED014E0FB
:100F580001F012FD38610AE001F00EFD02463B691E
:100F6800D31A41F28832934201D90323B5E03E4BAC
:100F78001B6F03F00203002BEED1FB7D012B05D183
:100F8800394B1B6C384A23F0805313647B689B6988
:100F9800002B00F0A180344B9B6803F00C03082B56
:100FA8005CD07B689B69022B41D1314B00221A60CF
:100FB80001F0E2FC386108E001F0DEFC02463B6922
:100FC800D31A022B01D9032387E0274B1B6803F0B0
:100FD8000073002BF0D17B68DA697B681B6A1A43BF
:100FE8007B685B6A9B011A437B689B6A5B08013BD1
:100FF8001B041A437B68DB6A1B061B4913434B60BF
:101008001B4B01221A6001F0B7FC386108E001F0BF
:10101800B3FC02463B69D31A022B01D903235CE0D7
:10102800114B1B6803F00073002BF0D054E0104BF9
:1010380000221A6001F0A0FC386108E001F09CFC75
:1010480002463B69D31A022B01D9032345E0064B1C
:101058001B6803F00073002BF0D13DE07B689B69AF
:10106800012B07D1012338E000380240007000400E
:10107800600047421B4B5B68FB607B689B69012BE8
:1010880028D0FB6803F480027B68DB699A4221D18F
:10109800FB6803F03F027B681B6A9A421AD1FA6820
:1010A80047F6C07313407A68526A9201934211D18D
:1010B800FB6803F440327B689B6A5B08013B1B04B6
:1010C8009A4207D1FB6803F070627B68DB6A1B06F3
:1010D8009A4201D0012300E0002318461837BD4684
:1010E80080BD00BF0038024080B584B000AF786092
:1010F80039607B68002B01D10123CCE0684B1B6869
:1011080003F007033A689A420CD9654B3A68D2B2A1
:101118001A70634B1B6803F007033A689A4201D0C0
:101128000123B8E07B681B6803F00203002B20D082
:101138007B681B6803F00403002B05D0594B9B68A0
:10114800584A43F4E05393607B681B6803F0080334
:10115800002B05D0534B9B68524A43F4604393607D
:10116800504B9B6823F0F0027B689B684D49134302
:101178008B607B681B6803F00103002B44D07B68FD
:101188005B68012B07D1474B1B6803F40033002B26
:1011980019D101237FE07B685B68022B03D07B6851
:1011A8005B68032B07D13F4B1B6803F00073002BD0
:1011B80009D101236FE03B4B1B6803F00203002BAE
:1011C80001D1012367E0374B9B6823F003027B685A
:1011D8005B68344913438B6001F0CEFBF8600AE08A
:1011E80001F0CAFB0246FB68D31A41F288329342E7
:1011F80001D903234FE02B4B9B6803F00C027B685B
:101208005B689B009A42EBD1254B1B6803F00703F0
:101218003A689A420CD2224B3A68D2B21A70204BE2
:101228001B6803F007033A689A4201D0012332E0B1
:101238007B681B6803F00403002B08D0194B9B68DC
:1012480023F4E0527B68DB68164913438B607B68A4
:101258001B6803F00803002B09D0124B9B6823F48A
:1012680060427B681B69DB000E4913438B6000F00A
:1012780021F802460B4B9B681B0903F00F030A4930
:10128800CB5C22FA03F3094A1360094B1B68184622
:1012980003F018FF002318461037BD4680BD00BF75
:1012A800003C024000380240646500083C00002011
:1012B800000000202DE9B04F94B000AF00237B64FC
:1012C8000023FB6400233B640023BB64794B9B68C9
:1012D80003F00C03082B0DD0082B00F2E180002B43
:1012E80002D0042B03D0DBE0734BBB64DBE0734B11
:1012F800BB64D8E06F4B5B6803F03F037B646D4BC6
:101308005B6803F48003002B63D06A4B5B689B091E
:101318000022BB63FA63BB6BC3F308033B63002380
:101328007B63D7E90C4522462B464FF000004FF06F
:101338000001590141EAD261500102460B4621469B
:10134800511A3961294663EB01037B614FF00002B2
:101358004FF00003D7E904AB59468B01514643EAE5
:10136800916351468A015146B2EB0108594663EB35
:1013780001094FF000024FF000034FEAC90343EAA6
:1013880058734FEAC80290469946234618EB030360
:10139800BB602B4649EB0303FB604FF000024FF0A4
:1013A8000003D7E9024529464B02214643EAD153B7
:1013B80021464A02104619467B6C0022BB62FA623B
:1013C800D7E90A23FEF7FCFE02460B461346FB64E8
:1013D80058E0384B5B689B09002218461146C0F359
:1013E80008033B6200237B62D7E9088942464B46E3
:1013F8004FF000004FF00001590141EAD26150015D
:1014080002460B464146B2EB010A494663EB010B23
:101418004FF000024FF000034FEA8B1343EA9A6340
:101428004FEA8A12B2EB0A0463EB0B054FF0000295
:101438004FF00003EB0043EA5473E20014461D46E4
:101448004346E3183B604B4645EB03037B604FF094
:1014580000024FF00003D7E9004529468B022146D8
:1014680043EA915321468A02104619467B6C0022B2
:10147800BB61FA61D7E90623FEF7A2FE02460B46D6
:101488001346FB640B4B5B681B0C03F0030301332F
:101498005B003B64FA6C3B6CB2FBF3F3BB6402E0A9
:1014A800054BBB6400BFBB6C18465037BD46BDE852
:1014B800B08F00BF003802400024F40000127A0008
:1014C80080B400AF034B1B681846BD465DF8047B2B
:1014D800704700BF3C00002080B500AFFFF7F0FF69
:1014E8000246054B9B689B0A03F007030349CB5C44
:1014F80022FA03F3184680BD0038024074650008DC
:1015080080B500AFFFF7DCFF0246054B9B685B0B1D
:1015180003F007030349CB5C22FA03F3184680BDA6
:10152800003802407465000880B483B000AF78606A
:1015380039607B680F221A60124B9B6803F0030224
:101548007B685A600F4B9B6803F0F0027B689A60D7
:101558000C4B9B6803F4E0527B68DA60094B9B688C
:10156800DB0803F4E0527B681A61074B1B6803F041
:1015780007023B681A6000BF0C37BD465DF8047B64
:10158800704700BF00380240003C024080B582B07E
:1015980000AF01F0F1F978605D4B1B685C4A43F0DD
:1015A8000103136008E001F0E7F902467B68D31AEB
:1015B800022B01D90323A7E0554B1B6803F0020354
:1015C800002BF0D0524B1B68514A43F08003136044
:1015D80001F0D2F978604E4B00229A600AE001F0DF
:1015E800CBF902467B68D31A41F28832934201D97B
:1015F800032389E0464B9B6803F00C03002BEED1D4
:1016080001F0BAF97860424B1B68414A23F4502331
:10161800136008E001F0B0F902467B68D31A642B26
:1016280001D9032370E03A4B1B6803F40033002B05
:10163800F0D101F0A1F97860354B1B68344A23F0EA
:101648008073136008E001F097F902467B68D31AAB
:10165800022B01D9032357E02D4B1B6803F00073BD
:10166800002BF0D101F088F97860294B1B68284AD3
:1016780023F08063136008E001F07EF902467B687E
:10168800D31A022B01D903233EE0214B1B6803F038
:101698000063002BF0D11E4B1E4A5A601C4B1E4A99
:1016A800C3F884201A4BDB68194A23F4F853D36033
:1016B800174BDB68164A23F40053D360144BDB68DE
:1016C800134A43F41F03D360114BDB68104A43F4F9
:1016D8000013D3600E4B5B6F0D4A23F00103536771
:1016E8000B4B5B6F0A4A43F0807353670B4B0C4AF2
:1016F8001A600C4B1B68184603F0E4FC0346002BE9
:1017080001D0012300E0002318460837BD4680BDFC
:101718000038024010300004003000203C00002057
:101728000024F4000000002080B586B000AFF86007
:10173800B960C7E900230123FB75234B1B7E012BEE
:1017480001D102233BE0204B01221A764CF25030A3
:1017580000F070F80346FB75FB7D002B2BD1FB686E
:10176800002B05D13B781946B86800F01BF916E044
:10177800FB68012B05D13B881946B86800F0EEF8E4
:101788000DE0FB68022B05D13B681946B86800F0EC
:10179800C3F804E0D7E90023B86800F08BF84CF2EE
:1017A800503000F047F80346FB75084B1B69074AA1
:1017B80023F001031361044B00221A76FB7D1846BF
:1017C8001837BD4680BD00BF5C000020003C0240C9
:1017D80080B483B000AF0023FB710B4B1B69002B57
:1017E8000BDA094B094A5A60074B094A5A60064BFB
:1017F8001B69002B01DA0123FB71FB7918460C37B2
:10180800BD465DF8047B7047003C024023016745F4
:10181800AB89EFCD80B400AF054B1B69044A43F098
:101828000043136100231846BD465DF8047B7047EA
:10183800003C024080B584B000AF78600023FB60B4
:101848001A4B0022DA6101F097F8F86010E07B6823
:10185800B3F1FF3F0CD07B68002B07D001F08CF868
:101868000246FB68D31A7A689A4201D2032319E028
:101878000F4BDB6803F48033002BE8D10C4BDB689B
:1018880003F00103002B02D0094B0122DA60084B58
:10189800DB6803F0F203002B03D000F0A5F8012366
:1018A80000E0002318461037BD4680BD5C000020CC
:1018B800003C024080B485B000AFF860C7E900235F
:1018C800144B1B69134A23F440731361114B1B69B2
:1018D800104A43F4407313610E4B1B690D4A43F0E1
:1018E80001031361FB683A681A60BFF36F8F00BF8A
:1018F800D7E900014FF000024FF000030A0000236F
:10190800F968043113460B6000BF1437BD465DF813
:10191800047B7047003C024080B483B000AF78601D
:1019280039600D4B1B690C4A23F4407313610A4B51
:101938001B69094A43F400731361074B1B69064A84
:1019480043F0010313617B683A681A6000BF0C37E3
:10195800BD465DF8047B7047003C024080B483B00C
:1019680000AF78600B467B800D4B1B690C4A23F453
:10197800407313610A4B1B69094A43F4807313616E
:10198800074B1B69064A43F0010313617B687A8899
:101998001A8000BF0C37BD465DF8047B704700BF56
:1019A800003C024080B483B000AF78600B46FB7007
:1019B8000C4B1B690B4A23F440731361094B094A0A
:1019C8001B691361074B1B69064A43F00103136146
:1019D8007B68FA781A7000BF0C37BD465DF8047B47
:1019E800704700BF003C024080B400AF274BDB6863
:1019F80003F01003002B08D0254BDB6943F01003DC
:101A0800234AD361214B1022DA60204BDB6803F0B4
:101A18002003002B08D01E4BDB6943F008031C4A47
:101A2800D3611A4B2022DA60184BDB6803F04003BD
:101A3800002B08D0164BDB6943F00403144AD3612A
:101A4800124B4022DA60114BDB6803F08003002B55
:101A580008D00F4BDB6943F002030D4AD3610B4BEF
:101A68008022DA60094BDB6803F00203002B08D000
:101A7800074BDB6943F02003054AD361034B02227D
:101A8800DA6000BFBD465DF8047B7047003C024049
:101A98005C00002080B485B000AF78600B46FB7016
:101AA8000023FB60FB78002B02D10023FB6010E0D1
:101AB800FB78012B03D14FF48073FB6009E0FB78BE
:101AC800022B03D14FF40073FB6002E04FF4407324
:101AD800FB60134B1B69124A23F440731361104BCC
:101AE8001A690F49FB6813430B610D4B1B690C4ABC
:101AF80023F0F80313610A4B1A697B68DB00134370
:101B0800074A43F002031361054B1B69044A43F477
:101B18008033136100BF1437BD465DF8047B7047FE
:101B2800003C024080B489B000AF7860396000237F
:101B38007B6100233B610023BB610023FB616BE1F8
:101B48000122FB6902FA03F37B613B681B687A692F
:101B580013403B613A697B699A4240F05A813B687D
:101B68005B6803F00303012B05D03B685B6803F057
:101B78000303022B30D17B689B68BB61FB695B0068
:101B8800032202FA03F3DB43BA691340BB613B68E3
:101B9800DA68FB695B0002FA03F3BA691343BB61B5
:101BA8007B68BA699A607B685B68BB610122FB69E4
:101BB80002FA03F3DB43BA691340BB613B685B6815
:101BC8001B0903F00102FB6902FA03F3BA69134324
:101BD800BB617B68BA695A603B685B6803F00303C2
:101BE800032B17D07B68DB68BB61FB695B000322B2
:101BF80002FA03F3DB43BA691340BB613B689A6896
:101C0800FB695B0002FA03F3BA691343BB617B68A3
:101C1800BA69DA603B685B6803F00303022B23D1DF
:101C2800FB69DA087B68083253F82230BB61FB692C
:101C380003F007039B000F2202FA03F3DB43BA69A0
:101C48001340BB613B681A69FB6903F007039B00FB
:101C580002FA03F3BA691343BB61FB69DA087B68CC
:101C68000832B96943F822107B681B68BB61FB69BD
:101C78005B00032202FA03F3DB43BA691340BB613A
:101C88003B685B6803F00302FB695B0002FA03F33D
:101C9800BA691343BB617B68BA691A603B685B68C1
:101CA80003F44033002B00F0B4800023FB60604B4A
:101CB8005B6C5F4A43F4804353645D4B5B6C03F495
:101CC8008043FB60FB685B4AFB699B08023352F860
:101CD8002330BB61FB6903F003039B000F2202FA68
:101CE80003F3DB43BA691340BB617B68524A9342F2
:101CF8002BD07B68514A934225D07B68504A934247
:101D08001FD07B684F4A934219D07B684E4A934252
:101D180013D07B684D4A93420DD07B684C4A93425E
:101D280007D07B684B4A934201D107230EE0082372
:101D38000CE006230AE0052308E0042306E0032359
:101D480004E0022302E0012300E00023FA6902F024
:101D5800030292009340BA691343BB613549FB699A
:101D68009B080233BA6941F823203B4B9B68BB614F
:101D78003B69DB43BA691340BB613B685B6803F4AA
:101D88008013002B03D0BA693B691343BB61324A05
:101D9800BB699360304BDB68BB613B69DB43BA6965
:101DA8001340BB613B685B6803F40013002B03D04E
:101DB800BA693B691343BB61274ABB69D360264BA9
:101DC8005B68BB613B69DB43BA691340BB613B6835
:101DD8005B6803F40033002B03D0BA693B691343F3
:101DE800BB611D4ABB6953601B4B1B68BB613B69E8
:101DF800DB43BA691340BB613B685B6803F480331B
:101E0800002B03D0BA693B691343BB61124ABB6913
:101E18001360FB690133FB61FB690F2B7FF690AE02
:101E280000BF00BF2437BD465DF8047B704700BF84
:101E3800003802400038014000000240000402401F
:101E480000080240000C024000100240001402404A
:101E580000180240001C0240003C014080B483B0DE
:101E680000AF78600B467B8013467B707B78002B35
:101E780003D07A887B689A6103E07B881A047B68C0
:101E88009A6100BF0C37BD465DF8047B704780B48B
:101E980085B000AF78600B467B807B685B69FB6030
:101EA8007A88FB6813401A04FB68D9437B880B4087
:101EB8001A437B689A6100BF1437BD465DF8047BFE
:101EC8007047000080B586B000AF786000237B6162
:101ED80000F052FD38617B68002B01D1012399E0A5
:101EE8007B68022283F835207B68002283F834203F
:101EF8007B681B681A687B681B6822F001021A60FD
:101F08000FE000F039FD02463B69D31A052B08D9CA
:101F18007B6820225A657B68032283F835200323D7
:101F280078E07B681B681B6803F00103002BE8D18D
:101F38007B681B681B687B617A69384B13407B613F
:101F48007B685A687B689B681A437B68DB681A431E
:101F58007B681B691A437B685B691A437B689B69CA
:101F68001A437B68DB691A437B681B6A13437A69E7
:101F780013437B617B685B6A042B07D17B68DA6A51
:101F88007B681B6B13437A6913437B617B681B680F
:101F98007A691A607B681B685B697B617B6923F0DF
:101FA80007037B617B685B6A7A6913437B617B68A3
:101FB8005B6A042B17D17B689B6A7A6913437B6140
:101FC8007B68DB6A002B0ED0786800F00DFB0346B7
:101FD800002B08D07B6840225A657B68012283F871
:101FE8003520012316E07B681B687A695A61786896
:101FF80000F0C4FA0346FB607B68DB6D3F229A4021
:10200800FB689A607B6800225A657B68012283F826
:102018003520002318461837BD4680BD3F8010F094
:1020280080B586B000AFF860B9607A603B60002385
:10203800FB75FB689B6D3B61FB6893F83430012BA3
:1020480001D1022340E0FB68012283F83420FB68B9
:1020580093F83530DBB2012B2FD1FB68022283F8CD
:102068003520FB6800225A653B687A68B968F868C9
:1020780000F056FAFB68DB6D3F229A403B699A6094
:10208800FB681B681A68FB681B6842F016021A6036
:10209800FB681B6C002B07D0FB681B681A68FB6881
:1020A8001B6842F008021A60FB681B681A68FB6824
:1020B8001B6842F001021A6005E0FB68002283F801
:1020C80034200223FB75FB7D18461837BD4680BDBA
:1020D80080B584B000AF78607B689B6DFB6000F0D2
:1020E8004BFCB8607B6893F83530DBB2022B08D024
:1020F8007B6880225A657B68002283F8342001239C
:1021080052E07B681B681A687B681B6822F016021D
:102118001A607B681B685A697B681B6822F080021A
:102128005A617B681B6C002B03D17B689B6C002B6E
:1021380007D07B681B681A687B681B6822F0080256
:102148001A607B681B681A687B681B6822F00102AA
:102158001A6013E000F010FC0246BB68D31A052B86
:102168000CD97B6820225A657B68032283F83520C6
:102178007B68002283F83420032315E07B681B6802
:102188001B6803F00103002BE4D17B68DB6D3F2261
:102198009A40FB689A607B68012283F835207B6847
:1021A800002283F83420002318461037BD4680BD2E
:1021B80080B483B000AF78607B6893F83530DBB2C9
:1021C800022B04D07B6880225A6501230CE07B68CF
:1021D800052283F835207B681B681A687B681B68B2
:1021E80022F001021A60002318460C37BD465DF83C
:1021F800047B704780B586B000AF78600023BB6071
:102208008E4B1B688E4AA2FB03239B0A7B617B686B
:102218009B6D3B613B691B68FB607B68DB6D08223B
:102228009A40FB681340002B1AD07B681B681B6818
:1022380003F00403002B13D07B681B681A687B68C3
:102248001B6822F004021A607B68DB6D08229A4042
:102258003B699A607B685B6D43F001027B685A6555
:102268007B68DB6D01229A40FB681340002B12D07B
:102278007B681B685B6903F08003002B0BD07B68CD
:10228800DB6D01229A403B699A607B685B6D43F085
:1022980002027B685A657B68DB6D04229A40FB6802
:1022A8001340002B12D07B681B681B6803F00203E5
:1022B800002B0BD07B68DB6D04229A403B699A6047
:1022C8007B685B6D43F004027B685A657B68DB6D55
:1022D80010229A40FB681340002B43D07B681B6890
:1022E8001B6803F00803002B3CD07B68DB6D1022D1
:1022F8009A403B699A607B681B681B6803F48023DB
:10230800002B18D07B681B681B6803F40023002B84
:1023180008D17B681B6C002B24D07B681B6C786809
:1023280098471FE07B689B6C002B1BD07B689B6CDD
:102338007868984716E07B681B681B6803F480730D
:10234800002B07D17B681B681A687B681B6822F022
:1023580008021A607B681B6C002B03D07B681B6C1F
:10236800786898477B68DB6D20229A40FB681340A9
:10237800002B00F08F807B681B681B6803F010033C
:10238800002B00F087807B68DB6D20229A403B6938
:102398009A607B6893F83530DBB2052B36D17B68C1
:1023A8001B681A687B681B6822F016021A607B6833
:1023B8001B685A697B681B6822F080025A617B6837
:1023C8001B6C002B03D17B689B6C002B07D07B68B0
:1023D8001B681A687B681B6822F008021A607B6811
:1023E800DB6D3F229A403B699A607B68012283F843
:1023F80035207B68002283F834207B681B6D002B16
:102408007ED07B681B6D7868984779E07B681B688D
:102418001B6803F48023002B1DD07B681B681B6896
:1024280003F40023002B0DD17B685B6C002B31D0AB
:102438007B685B6C786898472CE000BF3C00002004
:10244800B5814E1B7B68DB6B002B23D07B68DB6B75
:10245800786898471EE07B681B681B6803F48073E4
:10246800002B0FD17B681B681A687B681B6822F0F9
:1024780010021A607B68012283F835207B680022ED
:1024880083F834207B68DB6B002B03D07B68DB6B25
:10249800786898477B685B6D002B32D07B685B6DF2
:1024A80003F00103002B22D07B68052283F8352036
:1024B8007B681B681A687B681B6822F001021A6037
:1024C800BB680133BB607A699A4207D37B681B6893
:1024D8001B6803F00103002BF2D100E000BF7B680A
:1024E800012283F835207B68002283F834207B683A
:1024F800DB6C002B05D07B68DB6C7868984700E0C4
:1025080000BF1837BD4680BD80B483B000AF786087
:102518007B685B6D18460C37BD465DF8047B7047D9
:1025280080B485B000AFF860B9607A603B60FB6842
:102538001B681A68FB681B6822F480221A60FB6813
:102548001B683A685A60FB689B68402B08D1FB6897
:102558001B687A689A60FB681B68BA68DA6007E0EB
:10256800FB681B68BA689A60FB681B687A68DA605F
:1025780000BF1437BD465DF8047B704780B485B052
:1025880000AF78607B681B68DBB2103B144AA2FB83
:1025980003231B09FB60134AFB6813441B781A4684
:1025A8007B68DA65FB68032B09D97B681B6823F411
:1025B8007F7323F003031A1D7B689A6507E07B6825
:1025C8001B6823F47F7323F003037A6893657B68A1
:1025D8009B6D18461437BD465DF8047B704700BFF5
:1025E800ABAAAAAA5C63000880B485B000AF786083
:1025F8000023FB737B689B6ABB607B689B69002B2D
:102608001FD1BB68032B56D801A252F823F000BF94
:10261800292600083B26000829260008BF260008AE
:102628007B68DB6A03F08073002B46D00123FB73C1
:1026380043E07B68DB6AB3F1C07F40D10123FB73C1
:102648003DE07B689B69B3F5005F21D1BB68032B34
:1026580037D801A252F823F071260008772600081F
:1026680071260008892600080123FB7330E07B6887
:10267800DB6A03F08073002B25D00123FB7322E073
:102688007B68DB6AB3F1C07F1FD10123FB731CE0B9
:10269800BB68022B03D9BB68032B03D018E00123C6
:1026A800FB7315E07B68DB6A03F08073002B0ED0A8
:1026B8000123FB730BE000BF0AE000BF08E000BF86
:1026C80006E000BF04E000BF02E000BF00E000BF7A
:1026D800FB7B18461437BD465DF8047B704700BF86
:1026E80080B485B000AF78607B6803F00703FB60B7
:1026F8000C4BDB68BB60BA684FF6FF031340BB6046
:10270800FB681A02BB68134343F0BF6343F400330A
:10271800BB60044ABB68D36000BF1437BD465DF890
:10272800047B704700ED00E080B400AF044BDB6829
:102738001B0A03F007031846BD465DF8047B704783
:1027480000ED00E080B483B000AF0346FB7197F959
:102758000730002B0BDBFB7903F01F02074997F9C1
:1027680007305B09012000FA02F241F8232000BF7C
:102778000C37BD465DF8047B704700BF00E100E000
:1027880080B483B000AF03463960FB7197F9073016
:10279800002B0ADB3B68DAB20C4997F907301201C3
:1027A800D2B20B4483F800230AE03B68DAB2084946
:1027B800FB7903F00F03043B1201D2B20B441A76E3
:1027C80000BF0C37BD465DF8047B704700E100E0B0
:1027D80000ED00E080B489B000AFF860B9607A60BD
:1027E800FB6803F00703FB61FB69C3F10703042BD4
:1027F80028BF0423BB61FB690433062B02D9FB699C
:10280800033B00E000237B614FF0FF32BB6902FA13
:1028180003F3DA43BB681A407B699A404FF0FF31F3
:102828007B6901FA03F3D9437B680B4013431846CD
:102838002437BD465DF8047B704780B582B000AF91
:1028480078607868FFF74CFF00BF0837BD4680BD49
:1028580080B586B000AF0346B9607A60FB73002389
:102868007B61FFF761FF78617A68B9687869FFF77B
:10287800B1FF024697F90F3011461846FFF780FF5F
:1028880000BF1837BD4680BD80B582B000AF034693
:10289800FB7197F907301846FFF754FF00BF083758
:1028A800BD4680BD80B500AF0E4B1B680D4A43F492
:1028B800007313600B4B1B680A4A43F48063136070
:1028C800084B1B68074A43F4807313600320FFF723
:1028D800B4FF0F2002F0F6FB03F0B8F80023184607
:1028E80080BD00BF003C024080B500AF134B4FF0E5
:1028F800FF321A62114B00221A62104B4FF0FF325E
:102908005A620E4B00225A620C4B4FF0FF321A618A
:102918000A4B00221A61094B4FF0FF325A61074BEC
:1029280000225A61054B4FF0FF329A61034B002297
:102938009A6100F005F80023184680BD003802406F
:1029480080B400AF00BFBD465DF8047B704700004F
:1029580080B400AF064B1B781A46064B1B6813441D
:10296800044A136000BFBD465DF8047B704700BF92
:10297800040000207C00002080B400AF034B1B68DB
:102988001846BD465DF8047B704700BF7C000020F8
:1029980080B584B000AF7860FFF7EEFFB8607B6861
:1029A800FB60FB68B3F1FF3F05D00A4B1B781A4662
:1029B800FB681344FB6000BFFFF7DEFF0246BB68FD
:1029C800D31AFA689A42F7D800BF00BF1037BD463D
:1029D80080BD00BF0400002080B584B000AF7860DF
:1029E8007B68002B01D10123EDE07B6893F8203050
:1029F800DBB2002B02D1786803F0B8F87B681B685B
:102A08001A687B681B6842F001021A60FFF7B4FF7E
:102A1800F86012E0FFF7B0FF0246FB68D31A0A2BF2
:102A28000BD97B685B6A43F400327B685A627B6827
:102A3800052283F820200123C5E07B681B685B68BA
:102A480003F00103002BE5D07B681B681A687B68DC
:102A58001B6822F002021A60FFF78EFFF86012E08E
:102A6800FFF78AFF0246FB68D31A0A2B0BD97B684B
:102A78005B6A43F400327B685A627B68052283F8FC
:102A8800202001239FE07B681B685B6803F002033A
:102A9800002BE5D17B681B7E012B08D17B681B6866
:102AA8001A687B681B6842F080021A6007E07B683E
:102AB8001B681A687B681B6822F080021A607B68B2
:102AC8005B7E012B08D17B681B681A687B681B68D2
:102AD80042F040021A6007E07B681B681A687B684E
:102AE8001B6822F040021A607B689B7E012B08D18C
:102AF8007B681B681A687B681B6842F020021A60B2
:102B080007E07B681B681A687B681B6822F0200254
:102B18001A607B68DB7E012B08D17B681B681A680A
:102B28007B681B6822F010021A6007E07B681B684C
:102B38001A687B681B6842F010021A607B681B7F6A
:102B4800012B08D17B681B681A687B681B6842F0F8
:102B580008021A6007E07B681B681A687B681B68B4
:102B680022F008021A607B685B7F012B08D17B6822
:102B78001B681A687B681B6842F004021A6007E049
:102B88007B681B681A687B681B6822F004021A605D
:102B98007B689A687B68DB681A437B681B691A4301
:102BA8007B685B6942EA03017B685B685A1E7B6845
:102BB8001B680A43DA617B6800225A627B6801223B
:102BC80083F82020002318461037BD4680BD80B505
:102BD8008AB000AF786000237B627B681B685B6902
:102BE8003B627B681B685B68FB617B681B689B6852
:102BF800BB617B681B68DB687B617B681B681B6942
:102C08003B617B681B689B69FB603B6A03F00103BF
:102C1800002B7CD0BB6903F00103002B23D07B6819
:102C28001B6801229A60BB6903F00203002B03D0E2
:102C3800786800F083F916E0BB6903F00403002B01
:102C480004D07B6A43F400637B620CE0BB6903F049
:102C58000803002B04D07B6A43F480537B6202E0B4
:102C6800786800F089F9BB6903F48073002B24D0DD
:102C78007B681B684FF480729A60BB6903F4007329
:102C8800002B03D0786800F063F916E0BB6903F401
:102C98008063002B04D07B6A43F400537B620CE012
:102CA800BB6903F40063002B04D07B6A43F48043C0
:102CB8007B6202E0786800F069F9BB6903F480334D
:102CC800002B24D07B681B684FF480329A60BB6964
:102CD80003F40033002B03D0786800F043F916E0C2
:102CE800BB6903F48023002B04D07B6A43F40043C0
:102CF8007B620CE0BB6903F40023002B04D07B6AE1
:102D080043F480337B6202E0786800F049F93B6A5B
:102D180003F00803002B0CD07B6903F01003002B91
:102D280007D07B6A43F400737B627B681B681022C0
:102D3800DA603B6A03F00403002B0BD07B6903F0D5
:102D48000803002B06D07B681B680822DA607868C5
:102D580000F03AF93B6A03F00203002B09D07B68C4
:102D68001B68DB6803F00303002B02D0786800F0CF
:102D780021F93B6A03F04003002B0CD03B6903F0B8
:102D88001003002B07D07B6A43F480637B627B6867
:102D98001B6810221A613B6A03F02003002B0BD03A
:102DA8003B6903F00803002B06D07B681B680822E8
:102DB8001A61786800F01CF93B6A03F01003002BD5
:102DC80009D07B681B681B6903F00303002B02D042
:102DD800786800F003F93B6A03F40033002B0BD04A
:102DE800FB6903F01003002B06D07B681B681022D8
:102DF8005A60786800F006F93B6A03F48033002BC8
:102E08000BD0FB6903F00803002B06D07B681B6816
:102E180008225A60786800F0FFF83B6A03F4004320
:102E2800002B7BD0FB6903F00403002B72D03B6AB4
:102E380003F48073002B08D0FB6803F00103002B18
:102E480003D07B6A43F001037B623B6A03F400739F
:102E5800002B08D0FB6803F00203002B03D07B6A29
:102E680043F002037B623B6A03F48063002B08D0C3
:102E7800FB6803F00403002B03D07B6A43F00403D0
:102E88007B623B6A03F40063002B43D0FB6803F0CA
:102E98007003002B3ED0FB6803F07003602B2BD02F
:102EA800602B2ED8502B22D0502B2AD8402B19D04B
:102EB800402B26D8302B10D0302B22D8102B02D004
:102EC800202B05D01DE07B6A43F008037B6219E0E4
:102ED8007B6A43F010037B6214E07B6A43F02003B3
:102EE8007B620FE07B6A43F040037B620AE07B6A07
:102EF80043F080037B6205E07B6A43F480737B6266
:102F080000E000BF7B681B689A697B681B6822F039
:102F180070029A617B681B6804225A607B6A002BE6
:102F280008D07B685A6A7B6A1A437B685A62786859
:102F380000F07CF800BF2837BD4680BD80B483B060
:102F480000AF786000BF0C37BD465DF8047B704762
:102F580080B483B000AF786000BF0C37BD465DF821
:102F6800047B704780B483B000AF786000BF0C3733
:102F7800BD465DF8047B704780B483B000AF7860CD
:102F880000BF0C37BD465DF8047B704780B483B042
:102F980000AF786000BF0C37BD465DF8047B704712
:102FA80080B483B000AF786000BF0C37BD465DF8D1
:102FB800047B704780B483B000AF786000BF0C37E3
:102FC800BD465DF8047B704780B483B000AF78607D
:102FD80000BF0C37BD465DF8047B704780B483B0F2
:102FE80000AF786000BF0C37BD465DF8047B7047C2
:102FF80080B483B000AF786000BF0C37BD465DF881
:10300800047B704780B483B000AF786000BF0C3792
:10301800BD465DF8047B704780B483B000AF78602C
:1030280000BF0C37BD465DF8047B704780B483B0A1
:1030380000AF786000BF0C37BD465DF8047B704771
:1030480080B582B000AF78607B68002B01D1012386
:1030580041E07B6893F83D30DBB2002B06D17B68FA
:10306800002283F83C20786802F040FE7B68022248
:1030780083F83D207B681A687B680433194610463C
:1030880000F096FA7B68012283F846207B680122CB
:1030980083F83E207B68012283F83F207B68012269
:1030A80083F840207B68012283F841207B68012255
:1030B80083F842207B68012283F843207B68012241
:1030C80083F844207B68012283F845207B6801222D
:1030D80083F83D20002318460837BD4680BD000010
:1030E80080B485B000AF78607B6893F83D30DBB280
:1030F800012B01D001234EE07B68022283F83D209A
:103108007B681B68DA687B681B6842F00102DA603A
:103118007B681B68234A934222D07B681B68B3F103
:10312800804F1DD07B681B681F4A934218D07B686C
:103138001B681E4A934213D07B681B681C4A934243
:103148000ED07B681B681B4A934209D07B681B68BA
:10315800194A934204D07B681B68184A934211D1DC
:103168007B681B689B6803F00703FB60FB68062B02
:1031780010D07B681B681A687B681B6842F00102E4
:103188001A6007E07B681B681A687B681B6842F056
:1031980001021A60002318461437BD465DF8047B07
:1031A800704700BF000001400004004000080040D4
:1031B800000C00400004014000400140001800409D
:1031C80080B582B000AF78607B681B681B6903F02C
:1031D8000203022B22D17B681B68DB6803F0020321
:1031E800022B1BD17B681B686FF002021A617B6897
:1031F80001221A777B681B689B6903F00303002B85
:1032080003D0786800F0B5F905E0786800F0A7F910
:10321800786800F0B8F97B6800221A777B681B6829
:103228001B6903F00403042B22D17B681B68DB684D
:1032380003F00403042B1BD17B681B686FF00402A6
:103248001A617B6802221A777B681B689B6903F402
:103258004073002B03D0786800F08BF905E078689C
:1032680000F07DF9786800F08EF97B6800221A7703
:103278007B681B681B6903F00803082B22D17B6855
:103288001B68DB6803F00803082B1BD17B681B68ED
:103298006FF008021A617B6804221A777B681B6842
:1032A800DB6903F00303002B03D0786800F061F9B1
:1032B80005E0786800F053F9786800F064F97B68F5
:1032C80000221A777B681B681B6903F01003102B18
:1032D80022D17B681B68DB6803F01003102B1BD11D
:1032E8007B681B686FF010021A617B6808221A77E6
:1032F8007B681B68DB6903F44073002B03D0786894
:1033080000F037F905E0786800F029F9786800F0EE
:103318003AF97B6800221A777B681B681B6903F0FF
:103328000103012B0ED17B681B68DB6803F00103E6
:10333800012B07D17B681B686FF001021A6178685E
:1033480002F0D6FA7B681B681B6903F08003802BA8
:103358000ED17B681B68DB6803F08003802B07D1E4
:103368007B681B686FF080021A61786800F0E0FAE9
:103378007B681B681B6903F04003402B0ED17B68F8
:103388001B68DB6803F04003402B07D17B681B6890
:103398006FF040021A61786800F0FFF87B681B68DC
:1033A8001B6903F02003202B0ED17B681B68DB68A8
:1033B80003F02003202B07D17B681B686FF02002E5
:1033C8001A61786800F0AAFA00BF0837BD4680BDC8
:1033D80080B584B000AF786039600023FB737B68E8
:1033E80093F83C30012B01D10223B4E07B68012221
:1033F80083F83C207B68022283F83D207B681B68A9
:103408009B68BB60BB6823F07703BB60BB6823F491
:103418007F43BB607B681B68BA689A603B681B681F
:10342800B3F5005F3ED0B3F5005F00F28780B3F5D7
:10343800805F00F08680B3F5805F7FD8702B1AD04C
:10344800702B7BD8602B50D0602B77D8502B3CD07A
:10345800502B73D8402B58D0402B6FD8302B64D0CA
:10346800302B6BD8202B60D0202B67D8002B5CD05A
:10347800102B5AD062E07B6818683B6899683B68F3
:103488005A683B68DB6800F0ADF97B681B689B688D
:10349800BB60BB6843F07703BB607B681B68BA6896
:1034A8009A604FE07B6818683B6899683B685A687F
:1034B8003B68DB6800F096F97B681B689A687B6854
:1034C8001B6842F480429A603CE07B6818683B685D
:1034D80059683B68DB681A4600F00AF97B681B6884
:1034E8005021184600F063F92CE07B6818683B68A7
:1034F80059683B68DB681A4600F029F97B681B6845
:103508006021184600F053F91CE07B6818683B6896
:1035180059683B68DB681A4600F0EAF87B681B6864
:103528004021184600F043F90CE07B681A683B68B4
:103538001B681946104600F03AF903E00123FB73B3
:1035480000E000BF7B68012283F83D207B680022F1
:1035580083F83C20FB7B18461037BD4680BD80B4FD
:1035680083B000AF786000BF0C37BD465DF8047BC0
:10357800704780B483B000AF786000BF0C37BD4699
:103588005DF8047B704780B483B000AF786000BFFB
:103598000C37BD465DF8047B704780B483B000AF3C
:1035A800786000BF0C37BD465DF8047B70470000AB
:1035B80080B485B000AF786039607B681B68FB60B9
:1035C8007B68404A934213D07B68B3F1804F0FD099
:1035D8007B683D4A93420BD07B683C4A934207D0B4
:1035E8007B683B4A934203D07B683A4A934208D1AE
:1035F800FB6823F07003FB603B685B68FA68134361
:10360800FB607B682F4A93422BD07B68B3F1804FD5
:1036180027D07B682C4A934223D07B682B4A93425D
:103628001FD07B682A4A93421BD07B68294A934261
:1036380017D07B68284A934213D07B68274A934265
:103648000FD07B68264A93420BD07B68254A934269
:1036580007D07B68244A934203D07B68234A93426D
:1036680008D1FB6823F44073FB603B68DB68FA68A9
:103678001343FB60FB6823F080023B685B691343DC
:10368800FB607B68FA681A603B689A687B68DA6254
:103698003B681A687B689A627B680A4A934203D03F
:1036A8007B680C4A934203D13B681A697B681A63AA
:1036B8007B6801225A6100BF1437BD465DF8047B60
:1036C800704700BF000001400004004000080040AF
:1036D800000C00400004014000400140004401404B
:1036E8000048014000180040001C00400020004035
:1036F80080B487B000AFF860B9607A60FB681B6A75
:103708007B61FB681B6A23F00102FB681A62FB6895
:103718009B693B613B6923F0F0033B617B681B01BC
:103728003A6913433B617B6923F00A037B617A6939
:10373800BB6813437B61FB683A699A61FB687A69E5
:103748001A6200BF1C37BD465DF8047B704780B421
:1037580087B000AFF860B9607A60FB681B6A23F035
:103768001002FB681A62FB689B697B61FB681B6A35
:103778003B617B6923F470437B617B681B037A6937
:1037880013437B613B6923F0A0033B61BB681B01CA
:103798003A6913433B61FB687A699A61FB683A6945
:1037A8001A6200BF1C37BD465DF8047B704780B4C1
:1037B80085B000AF786039607B689B68FB60FB6808
:1037C80023F07003FB603A68FB68134343F0070378
:1037D800FB607B68FA689A6000BF1437BD465DF8E5
:1037E800047B704780B487B000AFF860B9607A6036
:1037F8003B60FB689B687B617B6923F47F437B614B
:103808003B681A027B681A43BB6813437A691343FF
:103818007B61FB687A699A6000BF1C37BD465DF81A
:10382800047B704780B485B000AF786039607B68EE
:1038380093F83C30012B01D102235AE07B68012226
:1038480083F83C207B68022283F83D207B681B6854
:103858005B68FB607B681B689B68BB60FB6823F048
:103868007003FB603B681B68FA681343FB607B6866
:103878001B68FA685A607B681B68214A934222D009
:103888007B681B68B3F1804F1DD07B681B681D4A9D
:10389800934218D07B681B681B4A934213D07B68FD
:1038A8001B681A4A93420ED07B681B68184A9342D9
:1038B80009D07B681B68174A934204D07B681B6851
:1038C800154A93420CD1BB6823F08003BB603B6868
:1038D8005B68BA681343BB607B681B68BA689A6008
:1038E8007B68012283F83D207B68002283F83C2016
:1038F800002318461437BD465DF8047B704700BFA7
:10390800000001400004004000080040000C004096
:1039180000040140004001400018004080B483B01A
:1039280000AF786000BF0C37BD465DF8047B704778
:1039380080B483B000AF786000BF0C37BD465DF837
:10394800047B704780B582B000AF78607B68002B3D
:1039580001D101233FE07B6893F83D30DBB2002BB7
:1039680006D17B68002283F83C20786802F00AFAC6
:103978007B68242283F83D207B681B68DA687B68B3
:103988001B6822F40052DA60786800F0FBFF7B685D
:103998001B681A697B681B6822F490421A617B686D
:1039A8001B685A697B681B6822F02A025A617B6887
:1039B8001B68DA687B681B6842F40052DA607B682F
:1039C80000221A647B68202283F83D207B6820222D
:1039D80083F83E20002318460837BD4680BD000006
:1039E80080B58CB000AFF860B9601346FB80FB6807
:1039F80093F83D30DBB2202B65D1BB68002B02D099
:103A0800FB88002B01D101235EE0FB6893F83C3072
:103A1800012B01D1022357E0FB68012283F83C20E7
:103A2800BA68FB681A62FB68FA889A84FB68FA88A5
:103A3800DA84FB6800221A64FB68212283F83D209F
:103A4800FB685B6B224ADA63FB685B6B214A1A648A
:103A5800FB685B6B204ADA64FB685B6B00221A65C3
:103A680007F10803FB62FB68586BFB6A1968FB687F
:103A78001B6804331A46FB88FEF7D2FAFB681B68FA
:103A88006FF040021A60FB68002283F83C20FB6854
:103A98001B681433BB61BB6953E8003F7B617B69DA
:103AA80043F08003BB62FB681B681433BA6A7A620E
:103AB8003B62396A7A6A41E80023FB61FB69002BA3
:103AC800E5D1002300E0022318463037BD4680BD0B
:103AD80025420008BF4200083744000880B584B07A
:103AE80000AFF860B9601346FB80FB6893F83E307E
:103AF800DBB2202B1DD1BB68002B02D0FB88002B2A
:103B080001D1012316E0FB6893F83C30012B01D169
:103B180002230FE0FB68012283F83C20FB680022A7
:103B28001A63FB881A46B968F86800F0CBFC0346AC
:103B380000E0022318461037BD4680BD80B59AB014
:103B480000AF78607B681B680C33BB64BB6C53E8C0
:103B5800003F7B647B6C23F490737B667B681B68F7
:103B68000C337A6E7A653B65396D7A6D41E80023CE
:103B7800FB64FB6C002BE5D17B681B6814337B630B
:103B88007B6B53E8003F3B633B6B23F001033B66D1
:103B98007B681B6814333A6E3A64FB63F96B3A6CC2
:103BA80041E80023BB63BB6B002BE5D17B681B6B33
:103BB800012B19D17B681B680C333B623B6A53E8C5
:103BC800003FFB61FB6923F01003FB657B681B6802
:103BD8000C33FA6DFA62BB62B96AFA6A41E80023EB
:103BE8007B627B6A002BE5D17B681B685B6903F00D
:103BF8004003402B36D17B681B681433FB60FB689D
:103C080053E8003FBB60BB6823F04003BB657B689B
:103C18001B681433BA6DBA617B617969BA6941E886
:103C280000233B613B69002BE5D17B689B6B002B34
:103C380018D07B689B6B00221A657B689B6B1846C3
:103C4800FEF746FA0346002B0CD07B689B6B1846A0
:103C5800FEF75AFC0346202B04D17B6810221A6415
:103C680003230AE07B680022DA857B68202283F838
:103C78003E207B6800221A63002318466837BD4639
:103C880080BD000080B5BAB000AF78607B681B6863
:103C98001B68C7F8E4307B681B68DB68C7F8E0304E
:103CA8007B681B685B69C7F8DC300023C7F8D8302D
:103CB8000023C7F8D430D7F8E43003F00F03C7F86F
:103CC800D830D7F8D830002B0FD1D7F8E43003F02C
:103CD8002003002B09D0D7F8E03003F02003002B95
:103CE80003D0786800F093FD56E2D7F8D830002B5F
:103CF80000F0DE80D7F8DC3003F00103002B06D19A
:103D0800D7F8E03003F49073002B00F0D180D7F897
:103D1800E43003F00103002B0BD0D7F8E03003F4B4
:103D28008073002B05D07B681B6C43F001027B6815
:103D38001A64D7F8E43003F00403002B0BD0D7F84B
:103D4800DC3003F00103002B05D07B681B6C43F0CB
:103D580002027B681A64D7F8E43003F00203002BF0
:103D68000BD0D7F8DC3003F00103002B05D07B68BB
:103D78001B6C43F004027B681A64D7F8E43003F044
:103D88000803002B11D0D7F8E03003F02003002BF4
:103D980005D1D7F8DC3003F00103002B05D07B6890
:103DA8001B6C43F008027B681A647B681B6C002B51
:103DB80000F0ED81D7F8E43003F02003002B08D0A1
:103DC800D7F8E03003F02003002B02D0786800F029
:103DD8001EFD7B681B685B6903F04003402B0CBF2A
:103DE80001230023DBB2C7F8D4307B681B6C03F0D7
:103DF8000803002B03D1D7F8D430002B4FD07868B4
:103E080000F026FC7B681B685B6903F04003402BCD
:103E180041D17B681B681433C7F89C30D7F89C30B5
:103E280053E8003FC7F89830D7F8983023F040039C
:103E3800C7F8D0307B681B681433D7F8D020C7F890
:103E4800A820C7F8A430D7F8A410D7F8A82041E8CC
:103E58000023C7F8A030D7F8A030002BD9D17B6851
:103E68009B6B002B13D07B689B6B7D4A1A657B6824
:103E78009B6B1846FEF79CF90346002B16D07B680F
:103E88009B6B1B6D7A68926B104698470EE07868BA
:103E980000F0AEF90AE0786800F0AAF906E0786860
:103EA80000F0A6F97B6800221A6470E100BF6EE199
:103EB8007B681B6B012B40F04A81D7F8E43003F094
:103EC8001003002B00F04381D7F8E03003F0100313
:103ED800002B00F03C810023BB607B681B681B68DB
:103EE800BB607B681B685B68BB60BB687B681B68E2
:103EF8005B6903F04003402B40F0B4807B689B6B08
:103F08001B685B68A7F8BE30B7F8BE30002B00F01E
:103F180040817B689B8DB7F8BE209A4280F039813A
:103F28007B68B7F8BE20DA857B689B6BDB69B3F5E5
:103F3800807F00F088807B681B680C33C7F8883066
:103F4800D7F8883053E8003FC7F88430D7F8843072
:103F580023F48073C7F8B8307B681B680C33D7F834
:103F6800B820C7F89420C7F89030D7F89010D7F841
:103F7800942041E80023C7F88C30D7F88C30002B08
:103F8800D9D17B681B6814337B677B6F53E8003F8C
:103F98003B673B6F23F00103C7F8B4307B681B68AD
:103FA8001433D7F8B420C7F88020FB67F96FD7F827
:103FB800802041E80023BB67BB6F002BE1D17B6801
:103FC8001B6814333B663B6E53E8003FFB65FB6D93
:103FD80023F04003C7F8B0307B681B681433D7F868
:103FE800B020FA66BB66B96EFA6E41E800237B66BC
:103FF8007B6E002BE3D17B68202283F83E207B6810
:1040080000221A637B681B680C33FB64FB6C53E863
:10401800003FBB64BB6C23F01003C7F8AC307B686F
:104028001B680C33D7F8AC20BA657B65796DBA6D1F
:1040380041E800233B653B6D002BE3D17B689B6B1C
:104048001846FEF745F87B689A8D7B68DB8D9BB236
:10405800D31A9BB21946786800F0D4F899E000BFEB
:104068001F4700087B689A8D7B68DB8D9BB2D31A4B
:10407800A7F8CE307B68DB8D9BB2002B00F08B80DD
:10408800B7F8CE30002B00F086807B681B680C33B5
:10409800BB63BB6B53E8003F7B637B6B23F490737C
:1040A800C7F8C8307B681B680C33D7F8C8207A6417
:1040B8003B64396C7A6C41E80023FB63FB6B002B93
:1040C800E3D17B681B6814337B627B6A53E8003F4B
:1040D8003B623B6A23F00103C7F8C4307B681B6866
:1040E8001433D7F8C4203A63FB62F96A3A6B41E8A3
:1040F8000023BB62BB6A002BE3D17B68202283F8D4
:104108003E207B6800221A637B681B680C333B6186
:104118003B6953E8003FFB60FB6823F01003C7F8D6
:10412800C0307B681B680C33D7F8C020FA61BB61CC
:10413800B969FA6941E800237B617B69002BE3D107
:10414800B7F8CE301946786800F05CF823E0D7F865
:10415800E43003F08003002B09D0D7F8E03003F0F7
:104168008003002B03D0786800F0E9FA14E0D7F850
:10417800E43003F04003002B0ED0D7F8E03003F012
:104188004003002B08D0786800F029FB04E000BF4A
:1041980002E000BF00E000BFE837BD4680BD00BFB9
:1041A80080B483B000AF786000BF0C37BD465DF8BF
:1041B800047B704780B483B000AF786000BF0C37D1
:1041C800BD465DF8047B704780B483B000AF78606B
:1041D80000BF0C37BD465DF8047B704780B483B0E0
:1041E80000AF786000BF0C37BD465DF8047B7047B0
:1041F80080B483B000AF786000BF0C37BD465DF86F
:10420800047B704780B483B000AF78600B467B8036
:1042180000BF0C37BD465DF8047B704780B590B091
:1042280000AF78607B689B6BFB637B681B681B68CF
:1042380003F48073002B37D1FB6B0022DA84FB6B0D
:104248001B6814337B627B6A53E8003F3B623B6A1E
:1042580023F08003BB63FB6B1B681433BA6B3A63B0
:10426800FB62F96A3A6B41E80023BB62BB6A002B28
:10427800E5D1FB6B1B680C333B613B6953E8003F9E
:10428800FB60FB6843F040037B63FB6B1B680C33EC
:104298007A6BFA61BB61B969FA6941E800237B610D
:1042A8007B69002BE5D102E0F86BFFF779FF00BFCF
:1042B8004037BD4680BD80B584B000AF78607B686C
:1042C8009B6BFB60F868FFF775FF00BF1037BD46B2
:1042D80080BD80B59CB000AF78607B689B6BFB6647
:1042E8007B681B681B6803F48073002B72D1FB6E1C
:1042F8000022DA85FB6E1B680C33FB64FB6C53E809
:10430800003FBB64BB6C23F48073BB66FB6E1B6809
:104318000C33BA6EBA657B65796DBA6D41E80023D6
:104328003B653B6D002BE5D1FB6E1B681433BB630B
:10433800BB6B53E8003F7B637B6B23F001037B6619
:10434800FB6E1B6814337A6E7A643B64396C7A6C42
:1043580041E80023FB63FB6B002BE5D1FB6E1B6878
:1043680014337B627B6A53E8003F3B623B6A23F06D
:1043780040033B66FB6E1B6814333A6E3A63FB627C
:10438800F96A3A6B41E80023BB62BB6A002BE5D1AE
:10439800FB6E202283F83E20FB6E1B6B012B19D18C
:1043A800FB6E1B680C333B613B6953E8003FFB60C5
:1043B800FB6823F01003FB65FB6E1B680C33FA6D7A
:1043C800FA61BB61B969FA6941E800237B617B69DD
:1043D800002BE5D1FB6E1B6B012B06D1FB6E9B8D71
:1043E8001946F86EFFF70EFF02E0F86EFFF7ECFED5
:1043F80000BF7037BD4680BD80B584B000AF78601F
:104408007B689B6BFB60FB681B6B012B08D1FB680F
:104418009B8D5B089BB21946F868FFF7F3FE02E034
:10442800F868FFF7DBFE00BF1037BD4680BD80B5DA
:1044380084B000AF78600023FB607B689B6BBB6037
:10444800BB681B685B6903F08003802B0CBF0123EA
:104458000023DBB2FB60BB6893F83D30DBB2212B55
:1044680008D1FB68002B05D0BB680022DA84B86845
:1044780000F0C6F8BB681B685B6903F04003402B7B
:104488000CBF01230023DBB2FB60BB6893F83E300E
:10449800DBB2222B08D1FB68002B05D0BB680022B9
:1044A800DA85B86800F0D4F8BB681B6C43F01002DA
:1044B800BB681A64B868FFF79BFE00BF1037BD469B
:1044C80080BD000080B598B000AFF860B9601346B1
:1044D800FB80BA68FB689A62FB68FA889A85FB6871
:1044E80000221A64FB68222283F83E20FB689B6B3B
:1044F800404ADA63FB689B6B3F4A1A64FB689B6B14
:104508003E4ADA64FB689B6B00221A6507F10803D0
:10451800FB65FB68986BFB681B6804331946FB6DE9
:104528001A68FB88FDF77CFD00233B61FB681B686C
:104538001B683B61FB681B685B683B613B69FB6808
:10454800002283F83C20FB681B69002B19D0FB680C
:104558001B680C333B643B6C53E8003FFB63FB6B0D
:1045680043F48073BB65FB681B680C33BA6DFA644F
:10457800BB64B96CFA6C41E800237B647B6C002B4C
:10458800E5D1FB681B681433FB62FB6A53E8003F04
:10459800BB62BB6A43F001037B65FB681B6814338D
:1045A8007A6DBA637B63796BBA6B41E800233B632E
:1045B8003B6B002BE5D1FB681B681433BB61BB69FF
:1045C80053E8003F7B617B6943F040033B65FB6830
:1045D8001B6814333A6D7A623B62396A7A6A41E839
:1045E8000023FB61FB69002BE5D1002318466037E7
:1045F800BD4680BDDB42000801440008374400087E
:1046080080B489B000AF78607B681B680C33FB60AE
:10461800FB6853E8003FBB60BB6823F0C003FB6145
:104628007B681B680C33FA69BA617B617969BA697E
:1046380041E800233B613B69002BE5D17B682022E0
:1046480083F83D2000BF2437BD465DF8047B7047E2
:1046580080B495B000AF78607B681B680C337B63CF
:104668007B6B53E8003F3B633B6B23F49073FB6425
:104678007B681B680C33FA6C3A64FB63F96B3A6C21
:1046880041E80023BB63BB6B002BE5D17B681B684B
:1046980014333B623B6A53E8003FFB61FB6923F03C
:1046A8000103BB647B681B681433BA6CFA62BB6293
:1046B800B96AFA6A41E800237B627B6A002BE5D17C
:1046C8007B681B6B012B19D17B681B680C33FB6063
:1046D800FB6853E8003FBB60BB6823F010037B64B2
:1046E8007B681B680C337A6CBA617B617969BA693B
:1046F80041E800233B613B69002BE5D17B68202220
:1047080083F83E207B6800221A6300BF5437BD46F9
:104718005DF8047B704780B584B000AF78607B6833
:104728009B6BFB60FB680022DA85FB680022DA8459
:10473800F868FFF75DFD00BF1037BD4680BD80B447
:1047480085B000AF78607B6893F83D30DBB2212BF1
:104758003ED17B689B68B3F5805F14D17B681B6989
:10476800002B10D17B681B6AFB60FB681B881A460C
:104778007B681B68C2F308025A607B681B6A9A1C34
:104788007B681A6208E07B681B6A591C7A681162A8
:104798001A787B681B685A607B68DB8C9BB2013B8C
:1047A8009BB27A681946D184002B0FD17B681B68AD
:1047B800DA687B681B6822F08002DA607B681B6815
:1047C800DA687B681B6842F04002DA60002300E088
:1047D800022318461437BD465DF8047B704780B540
:1047E80082B000AF78607B681B68DA687B681B68FA
:1047F80022F04002DA607B68202283F83D20786846
:10480800FFF7CEFC002318460837BD4680BD80B5AB
:104818008CB000AF78607B6893F83E30DBB2222B17
:1048280040F0AB807B689B68B3F5805F17D17B68ED
:104838001B69002B13D10023FB627B689B6ABB6258
:104848007B681B685B689BB2C3F308039AB2BB6AB8
:104858001A807B689B6A9A1C7B689A6226E07B6850
:104868009B6AFB620023BB627B689B68B3F5805F31
:1048780007D07B689B68002B0AD17B681B69002BDB
:1048880006D17B681B685B68DAB2FB6A1A7008E0BD
:104898007B681B685B68DBB203F07F03DAB2FB6AF4
:1048A8001A707B689B6A5A1C7B689A627B68DB8DEE
:1048B8009BB2013B9BB27A681946D185002B5AD12D
:1048C8007B681B68DA687B681B6822F02002DA6064
:1048D8007B681B68DA687B681B6822F48072DA6080
:1048E8007B681B685A697B681B6822F001025A6161
:1048F8007B68202283F83E207B681B6B012B35D117
:104908007B6800221A637B681B680C337B617B69B8
:1049180053E8003F3B613B6923F010037B627B68EF
:104928001B680C337A6A3A62FB61F9693A6A41E8B2
:104938000023BB61BB69002BE5D17B681B681B6842
:1049480003F01003102B0AD10023FB607B681B685F
:104958001B68FB607B681B685B68FB60FB687B68A7
:104968009B8D19467868FFF74DFC02E07868FFF7E1
:104978002BFC002302E0002300E002231846303716
:10498800BD4680BD2DE9B04FC0B000AFC7F8F400F8
:10499800D7F8F4301B681B6923F44050D7F8F4307B
:1049A800D968D7F8F4301A6840EA01031361D7F8D8
:1049B800F4309A68D7F8F4301B691A43D7F8F43002
:1049C8005B691A43D7F8F430DB691343C7F8F8304A
:1049D800D7F8F4301B68DB6823F4164121F00C018A
:1049E800D7F8F4301A68D7F8F8300B43D360D7F803
:1049F800F4301B685B6923F44070D7F8F430996988
:104A0800D7F8F4301A6840EA01035361D7F8F43054
:104A18001A688F4B9A4205D0D7F8F4301A688D4B34
:104A28009A4204D1FCF76CFDC7F8FC0003E0FCF7E0
:104A380053FDC7F8FC00D7F8F430DB69B3F5004F35
:104A480040F00C81D7F8FC300022C7F8E830C7F8EE
:104A5800EC20D7E93A4522462B469118B9655B41C7
:104A6800FB65D7E91623214612EB0108294643EBDB
:104A780001094FF000024FF000034FEAC90343EA6F
:104A880058734FEAC80290469946234618EB030329
:104A9800C7F8E0302B4649EB0303C7F8E430D7F8F2
:104AA800F4305B680022C7F8D830C7F8DC20D7E9B3
:104AB80036120B46DB183B65134642EB03037B6556
:104AC800D7E91423D7E93801FBF77AFB02460B46EE
:104AD800614BA3FB02235B091C01D7F8FC300022C1
:104AE800C7F8D030C7F8D420D7E9348942464B46B6
:104AF8009118B9645B41FB64D7E91223414612EB74
:104B0800010A494643EB010B4FF000024FF0000346
:104B18004FEACB0343EA5A734FEACA0292469B46CE
:104B280043461AEB0303C7F8C8304B464BEB030365
:104B3800C7F8CC30D7F8F4305B680022C7F8C0302B
:104B4800C7F8C420D7E930120B46DB183B6413467C
:104B580042EB03037B64D7E91023D7E93201FBF763
:104B68002FFB02460B4611463B4BA3FB01235B0977
:104B7800642202FB03F3CB1ADB0003F13202364B4B
:104B8800A3FB02235B095B0003F4F8731C44D7F80A
:104B9800FC300022C7F8B830C7F8BC20D7E92E8906
:104BA80042464B469118B9635B41FB63D7E90E2334
:104BB80041465118396349464B417B634FF0000227
:104BC8004FF00003D7E90CAB5946CB00514643EAF6
:104BD80051735146CA0010461946034642469B186F
:104BE800C7F8B0304B460A4642EB0303C7F8B43067
:104BF800D7F8F4305B680022C7F8A830C7F8AC20B3
:104C0800D7E92A120B46DB18BB62134642EB0303B3
:104C1800FB62D7E90A23D7E92C01FBF7D1FA024650
:104C28000B460D4BA3FB02135B09642101FB03F345
:104C3800D31ADB003233084AA2FB03235B0903F0D3
:104C48000702D7F8F4301B6822449A6005E100BFD8
:104C580000100140001401401F85EB51D7F8FC30CB
:104C68000022C7F8A030C7F8A420D7E9288942460F
:104C78004B46911839625B417B62D7E9082341466C
:104C88005418494643EB01054FF000024FF000036A
:104C9800EB0043EA5473E20014461D464346E3180A
:104CA800C7F898304B4645EB0303C7F89C30D7F854
:104CB800F4305B680022C7F89030C7F894204FF0B2
:104CC80000024FF00003D7E9244529468B0021460E
:104CD80043EA917321468A00D7E92601FBF770FA67
:104CE80002460B46604BA3FB02235B091C01D7F865
:104CF800FC300022C7F88830C7F88C20D7E9228911
:104D080042464B469118B9615B41FB61D7E90623DE
:104D180041465118396149464B417B614FF00002C9
:104D28004FF00003D7E904AB5946CB00514643EA9C
:104D380051735146CA0010461946034642469B180D
:104D4800C7F880304B460A4642EB0303C7F8843065
:104D5800D7F8F4305B680022BB67FA674FF00002AF
:104D68004FF00003D7E91E8949468B00414643EAC4
:104D7800917341468A00D7E92001FBF721FA0246E0
:104D88000B46394BA3FB02135B09642101FB03F3B8
:104D9800D31A1B013233344AA2FB03235B0903F005
:104DA800F0031C44D7F8FC3000223B677A67D7E948
:104DB8001C8942464B469118B9605B41FB60D7E9B4
:104DC800022341465118396049464B417B604FF0F8
:104DD80000024FF00003D7E900AB5946CB0051461B
:104DE80043EA51735146CA001046194603464246E3
:104DF8009B18BB664B460A4642EB0303FB66D7F893
:104E0800F4305B6800223B667A664FF000024FF090
:104E18000003D7E9188949468B00414643EA917354
:104E280041468A00D7E91A01FBF7CAF902460B4640
:104E38000D4BA3FB02135B09642101FB03F3D31A97
:104E48001B013233084AA2FB03235B0903F00F025C
:104E5800D7F8F4301B6822449A6000BF07F58077C2
:104E6800BD46BDE8B08F00BF1F85EB5180B485B04B
:104E780000AF78600B467B80FF23FB73FF23BB7377
:104E880013E07B685A1C7A601A78BB7B5340DBB20C
:104E9800BB600F4ABB6813441A78FB7B5340BB7353
:104EA8000C4ABB6813441B78FB737B885A1E7A80B4
:104EB800002BE6D1FB7B1B021AB2BB7B1BB2134350
:104EC8001BB29BB218461437BD465DF8047B704789
:104ED800646300086464000880B485B000AF78603B
:104EE8000023FB607B68B3F1006F03D37B68B3F1E9
:104EF800016F02D94FF0FF331BE00023BB6014E0C1
:104F08000F4ABB6852F823307A689A420AD3BB68C2
:104F180001330B4A52F823307A689A4202D2BB68AE
:104F2800FB6005E0BB680133BB60BB68072BE7DDAE
:104F3800FB6818461437BD465DF8047B704700BF10
:104F480008000020B0B586B000AFF860B96013461D
:104F5800FB8000237B7572B600BFFCF739FC254B3C
:104F6800F322DA60F868FFF7B7FF03467B757B7DAD
:104F7800214A92F90020934208D07B7D02211846ED
:104F8800FCF788FD97F915201B4B1A7000237B82CC
:104F98000023FB8221E0FB8A5B00BA6813441B886C
:104FA8007B82FB8A5B001A46FB68D1187B8A002249
:104FB8001C46154622462B460120FCF7B5FB034646
:104FC8007B747B7C002B05D0FCF724FC62B600BF09
:104FD80002230BE0FB8A0133FB82FA8AFB889A42A0
:104FE800D9D3FCF717FC62B600BF0323184618375D
:104FF800BD46B0BD003C02403800002080B582B0FC
:1050080000AF0023FB7172B600BFFCF7E1FB124B47
:10501800F322DA601148FFF75FFF0346FB71FB7963
:1050280002211846FCF736FD4FF00F024FF000033F
:105038000A490120FCF778FB0346BB71FCF7EAFB41
:1050480062B600BFBB79002B01D1012300E0002329
:1050580018460837BD4680BD003C02400080000865
:1050680080B487B000AFF860B9607A6000237B61D4
:1050780000237B82FB681B889AB2BB681A80BB68D6
:105088001B887B827B6901337B617B8A18461C37CE
:10509800BD465DF8047B704780B582B000AF002341
:1050A800FB8000233B603B46012219460448FFF77A
:1050B800D7FF0346FB80FB8818460837BD4680BDEE
:1050C8000080000880B58CB000AF78600023BB6218
:1050D80000237B620023BB602F4B5B6C2E4A43F49A
:1050E800803353642C4B5B6C03F48033BB60BB6828
:1050F80007F10C0207F1100311461846FCF714FAE1
:10510800FCF7FEF903465B00BB62BB6A234AA2FBBD
:1051180003239B0C013B7B62214B224A1A60204BE4
:1051280040F2E732DA601E4A7B6A53601C4B002269
:105138001A611B4B00229A60194B00229A61184889
:10514800FDF77EFF034687F82F3097F82F30002BA6
:105158001BD11348FDF7C4FF034687F82F3097F893
:105168002F30002B11D11820FDF78EFB7B680F2BF9
:1051780008D8002279681820FDF76AFB0A4A7B687C
:10518800136002E0012387F82F3097F82F30184674
:105198003037BD4680BD00BF0038024083DE1B4368
:1051A80080000020004001400000002080B584B04D
:1051B80000AFFDF777FB00F08DF800F0EDFA00F096
:1051C800C3FA00F0F1F800F041F900F0ABF900F093
:1051D80073F900F0F3F900F03FFA00F08BFA334B63
:1051E8004FF000629A60324B1B68DA68304B1B68DC
:1051F80042F01002DA604FF480722E492C48FEF714
:105208006DFC2B4B1B685A69294B1B6842F0010245
:105218005A61FFF741FF03469AB2274B1A80264B83
:105228001B884AF6CD32934201D100F061FF234B2F
:105238001B78002B05D1204B1B884AF6CD329342B0
:105248001FD072B600BF1E4B1B681E4A934216D869
:105258001B4B1B68B3F1005F11D3FDF745FBFCF74F
:1052680095F9194B1B68FB60FB68BB60144B1B6806
:105278007B607B6883F3088800BFBB68984762B689
:1052880000BFFDF779FB0246104B1B68D31AB3F534
:105298007A7FC4D94FF4A0510D48FCF7F8FDFDF70B
:1052A8006BFB0346094A1360B9E700BF00ED00E055
:1052B80038020020480300203C0300209405002009
:1052C8000000020800000220040002084003002039
:1052D8000008024080B594B000AF07F120033022E7
:1052E8000021184601F022F807F10C0300221A6089
:1052F8005A609A60DA601A610023BB60284B1B6C05
:10530800274A43F080531364254B1B6C03F08053EA
:10531800BB60BB6800237B60224B1B68214A43F4B7
:10532800804313601F4B1B6803F480437B607B68DA
:1053380001233B624FF480337B620223BB634FF44B
:105348008003FB6304233B6490237B640223BB64D8
:105358000423FB6407F120031846FBF74DFC0346C2
:10536800002B01D000F0D6FA0F23FB6002233B612B
:1053780000237B614FF4A053BB614FF48053FB6162
:1053880007F10C0304211846FBF7AEFE0346002B79
:1053980001D000F0BFFA00BF5037BD4680BD00BF46
:1053A800003802400070004080B584B000AF3B4632
:1053B80000221A605A609A60DA60214B214A1A600A
:1053C8001F4B00225A601E4B00229A601C4B002281
:1053D8001A611B4B00221A76194B002283F82020F1
:1053E800174B0022DA62164B174A9A62144B0022B6
:1053F800DA60134B0122DA61114B002283F8302066
:105408000F4B01225A610E48FBF75CF80346002B4C
:1054180001D000F07FFA04233B6001237B60002366
:10542800BB603B4619460648FBF7BEF90346002B0E
:1054380001D000F06FFA00BF1037BD4680BD00BF35
:10544800C8000020002001400100000F80B500AF17
:10545800174B184A1A60164B03225A60144B002245
:105468009A60134B0022DA60114B4FF400221A6144
:105478000F4B4FF480125A610D4B00221A760C4BD9
:1054880001225A760A4B00229A76094B0022DA76D4
:10549800074B00221A77064B01225A770448FDF77A
:1054A8009BFA0346002B01D000F034FA00BF80BD00
:1054B800100100200064004080B500AF174B184A67
:1054C8001A60164B03225A60144B00229A60134B41
:1054D8000022DA60114B4FF400221A610F4B4FF48F
:1054E80080125A610D4B00221A760C4B01225A7613
:1054F8000A4B00229A76094B0022DA76074B0022E3
:105508001A77064B01225A770448FDF765FA0346D5
:10551800002B01D000F0FEF900BF80BD380100204B
:105528000068004080B586B000AF07F1080300228C
:105538001A605A609A60DA603B4600221A605A6024
:105548001D4B4FF080421A601B4B47225A601A4B82
:1055580000229A60184B44F61F62DA60164B00224C
:105568001A61154B00229A611348FDF769FD03463D
:10557800002B01D000F0CEF94FF48053BB6007F147
:10558800080319460C48FDF723FF0346002B01D0FA
:1055980000F0C0F900233B6000237B603B461946BE
:1055A8000548FEF73FF90346002B01D000F0B2F999
:1055B80000BF1837BD4680BD6001002080B586B0A9
:1055C80000AF07F1080300221A605A609A60DA6097
:1055D8003B4600221A605A601D4B1E4A1A601C4B3B
:1055E80047225A601A4B00229A60194B41F61F4213
:1055F800DA60174B00221A61154B00229A61144891
:10560800FDF71EFD0346002B01D000F083F94FF48F
:105618008053BB6007F1080319460D48FDF7D8FE13
:105628000346002B01D000F075F900233B600023EE
:105638007B603B4619460648FEF7F4F80346002B04
:1056480001D000F067F900BF1837BD4680BD00BF24
:10565800A80100200004004080B586B000AF07F123
:10566800080300221A605A609A60DA603B460022FA
:105678001A605A601D4B1E4A1A601C4B47225A601A
:105688001A4B00229A60194B41F61F42DA60174BF9
:1056980000221A61154B00229A611448FDF7D0FCCC
:1056A8000346002B01D000F035F94FF48053BB605E
:1056B80007F1080319460D48FDF78AFE0346002B3B
:1056C80001D000F027F900233B6000237B603B46B4
:1056D80019460648FEF7A6F80346002B01D000F04D
:1056E80019F900BF1837BD4680BD00BFF001002082
:1056F8000008004080B500AF114B124A1A60104BE9
:105708004FF4E1325A600E4B00229A600C4B002293
:10571800DA600B4B00221A61094B0C225A61084BC4
:1057280000229A61064B0022DA610548FEF70AF961
:105738000346002B01D000F0EDF800BF80BD00BF8C
:10574800380200200010014080B582B000AF00236D
:105758007B60104B1B6B0F4A43F4800313630D4BA4
:105768001B6B03F480037B607B68002200213A20D6
:10577800FDF76EF83A20FDF787F800220021462051
:10578800FDF766F84620FDF77FF800BF0837BD46ED
:1057980080BD00BF0038024080B58AB000AF07F175
:1057A800140300221A605A609A60DA601A610023B2
:1057B8003B614B4B1B6B4A4A43F080031363484BD6
:1057C8001B6B03F080033B613B690023FB60444B88
:1057D8001B6B434A43F004031363414B1B6B03F0F9
:1057E8000403FB60FB680023BB603D4B1B6B3C4A1A
:1057F80043F0010313633A4B1B6B03F00103BB60D7
:10580800BB6800237B60364B1B6B354A43F00203B1
:105818001363334B1B6B03F002037B607B6800222E
:1058280040F201212F48FCF719FB01224FF4E05107
:105838002C48FCF713FB0022C7212B48FCF70EFB72
:105848000022C0212948FCF709FB41F601637B616E
:105858000123BB610023FB6100233B6207F11403B2
:1058680019462048FCF75EF9C7237B610123BB6119
:105878000023FB6100233B6207F1140319461A4811
:10588800FCF750F94FF480737B610023BB61002360
:10589800FB6107F1140319461348FCF743F9C023C9
:1058A8007B610123BB610023FB6100233B6207F19D
:1058B800140319460D48FCF735F9002203210A485C
:1058C800FCF7CCFA0022C0210748FCF7C7FA0022EF
:1058D800C0210648FCF7C2FA00BF2837BD4680BD84
:1058E8000038024000080240000002400004024064
:1058F80080B582B000AF78607B681B68044A934229
:1059080001D1FDF725F800BF0837BD4680BD00BFAF
:105918000040014080B400AF72B600BFFEE780B41B
:1059280000AFFEE780B400AFFEE780B400AFFEE74B
:1059380080B400AFFEE780B400AF00BFBD465DF89D
:10594800047B704780B400AF00BFBD465DF8047BA0
:10595800704780B400AF00BFBD465DF8047B704758
:1059680080B400AF00BFBD465DF8047B70470000FF
:1059780080B500AF0248FAF7E8FD00BF80BD00BF60
:10598800C800002080B500AF0248FDF720F900BF2D
:1059980080BD00BF1001002080B500AF0248FDF7B0
:1059A80016F900BF80BD00BF1001002080B500AF10
:1059B8000248FDF705FC00BF80BD00BF8000002045
:1059C80080B500AF0348FEF75DF9024800F0B2FA6F
:1059D80000BF80BD3802002080B500AF0248FCF748
:1059E80009FC00BF80BD00BF7C02002080B500AF6D
:1059F8000248FDF7ECF800BF80BD00BF3801002069
:105A080080B500AF0248FDF7E2F800BF80BD00BFD7
:105A18003801002080B500AF0248FCF7EBFB00BF5F
:105A280080BD00BFDC02002080B400AF064BD3F875
:105A38008830054A43F47003C2F8883000BFBD4679
:105A48005DF8047B704700BF00ED00E080B483B0D0
:105A580000AF00237B60104B5B6C0F4A43F480431C
:105A680053640D4B5B6C03F480437B607B680023BD
:105A78003B60094B1B6C084A43F080531364064B88
:105A88001B6C03F080533B603B6800BF0C37BD467E
:105A98005DF8047B704700BF0038024080B58AB0CB
:105AA80000AF786007F1140300221A605A609A6008
:105AB800DA601A617B681B68284A934249D100233F
:105AC8003B61274B5B6C264A43F480735364244B39
:105AD8005B6C03F480733B613B690023FB60204BE4
:105AE8001B6B1F4A43F0010313631D4B1B6B03F031
:105AF8000103FB60FB680023BB60194B1B6B184A52
:105B080043F002031363164B1B6B03F00203BB60E5
:105B1800BB6810237B610323BB610023FB6107F192
:105B2800140319460F48FBF7FDFF03237B6103238A
:105B3800BB610023FB6107F1140319460A48FBF710
:105B4800F1FF002200211220FCF782FE1220FCF750
:105B58009BFE00BF2837BD4680BD00BF0020014026
:105B680000380240000002400004024080B58CB0BA
:105B780000AF786007F11C0300221A605A609A602F
:105B8800DA601A617B681B68534A934246D1534BCB
:105B98001B680133514A1360504B1B68012B0DD110
:105BA8000023BB614E4B1B6C4D4A43F000731364DA
:105BB8004B4B1B6C03F00073BB61BB6900237B611B
:105BC800474B1B6B464A43F002031363444B1B6B62
:105BD80003F002037B617B694FF44073FB6102238E
:105BE8003B6200237B620323BB620923FB6207F14C
:105BF8001C0319463B48FBF795FF0022002114209F
:105C0800FCF726FE1420FCF73FFE00220021162098
:105C1800FCF71EFE1620FCF737FE58E07B681B6871
:105C2800314A934253D100233B612D4B1B6C2C4AC4
:105C380043F0806313642A4B1B6C03F080633B6161
:105C48003B69264B1B680133244A1360234B1B68AE
:105C5800012B0DD10023FB60214B1B6C204A43F024
:105C6800007313641E4B1B6C03F00073FB60FB682E
:105C78000023BB601A4B1B6B194A43F002031363E2
:105C8800174B1B6B03F00203BB60BB684FF4405318
:105C9800FB6102233B6200237B620323BB6209236F
:105CA800FB6207F11C0319460E48FBF73BFF002275
:105CB80000214020FCF7CCFD4020FCF7E5FD002248
:105CC80000214220FCF7C4FD4220FCF7DDFD00BFA7
:105CD8003037BD4680BD00BF00640040440300204B
:105CE80000380240000402400068004080B487B0D9
:105CF80000AF78607B681B68B3F1804F0ED100233A
:105D08007B611D4B1B6C1C4A43F0010313641A4B47
:105D18001B6C03F001037B617B6926E07B681B68D1
:105D2800164A93420ED100233B61134B1B6C124A57
:105D380043F002031364104B1B6C03F002033B6136
:105D48003B6912E07B681B680D4A93420DD1002322
:105D5800FB60094B1B6C084A43F004031364064BB1
:105D68001B6C03F00403FB60FB6800BF1C37BD46D7
:105D78005DF8047B704700BF003802400004004013
:105D88000008004080B58AB000AF786007F11403BE
:105D980000221A605A609A60DA601A617B681B6890
:105DA8004C4A934240F0928000233B614A4B5B6C23
:105DB800494A43F010035364474B5B6C03F01003EC
:105DC8003B613B690023FB60434B1B6B424A43F03A
:105DD80001031363404B1B6B03F00103FB60FB687B
:105DE8004FF4C0637B610223BB610023FB61032383
:105DF8003B6207237B6207F1140319463748FBF718
:105E080091FE374B374A1A60354B4FF000625A60A3
:105E1800334B00229A60324B0022DA60304B4FF449
:105E280080621A612E4B00225A612D4B00229A6122
:105E38002B4B4FF48072DA61294B00221A62284BEF
:105E480000225A622648FCF73DF80346002B01D091
:105E5800FFF760FD7B68224A9A63214A7B68936357
:105E6800214B224A1A60204B4FF000625A601E4BA9
:105E780040229A601C4B0022DA601B4B4FF4806270
:105E88001A61194B00225A61174B00229A61164B6E
:105E98000022DA61144B00221A62134B00225A6264
:105EA8001148FCF70FF80346002B01D0FFF732FD2D
:105EB8007B680D4A5A630C4A7B6893630022002171
:105EC8002520FCF7C5FC2520FCF7DEFC00BF2837A1
:105ED800BD4680BD0010014000380240000002406D
:105EE8007C02002040640240DC020020B8640240CA
:105EF80080B582B000AF78600B46FB70FCF73CFDC4
:105F080003460A4A136000BFFCF736FD0246074BFA
:105F18001B689A42F8D0FB789BB21A467968044805
:105F2800FDF75EFD00BF0837BD4680BD980500201F
:105F38003802002080B584B000AF78600023FB6091
:105F48007B68244A934240D17B681B681B6803F036
:105F58001003102B39D10023BB607B681B681B68BA
:105F6800BB607B681B685B68BB60BB687868FDF7D3
:105F7800E5FD7B689B6B1B685B68C3F58073FB6002
:105F8800154B1B78FE2B14D1134B1B79CC2B10D13E
:105F9800124B93F8003183F00103DBB2002B08D0D9
:105FA800FA680D490D4800F0B3F90C4B012283F84B
:105FB80000214FF480720021074800F0B7F94FF430
:105FC800807205497868FDF789FD00BF1037BD4626
:105FD80080BD00BF3802002048030020480400208C
:105FE80080B584B000AF03463960FB710023FB60C5
:105FF800FB685A1CFA602D4AFE21D154FB685A1CD2
:10600800FA602A4A0021D154FB685A1CFA60274AD0
:106018000021D154FB685A1CFA60244A0021D1544B
:10602800FB685A1CFA60214ACC21D154FB685A1CDF
:10603800FA601E4A1521D154FB685A1CFA601B49A4
:10604800FA79CA54FB685A1CFA603A681178174AF8
:10605800D154FB685A1CFA603A685178134AD154F3
:10606800FB685A1CFA60114A0121D154FB68DBB263
:10607800063BDAB20D4B5A70FB689BB219460B48C7
:10608800FEF7F4FE03467B81FB68084A13447A89CD
:106098001A80FB680233FB60FB68DBB219460348D1
:1060A800FFF726FF00BF1037BD4680BD4C05002016
:1060B80080B400AF0D4B93F83D30DBB2202B0DD1EF
:1060C8000A4B1B681B6803F04003402B06D1074BA3
:1060D8001B681B6803F08003802B01D0002300E0BD
:1060E80001231846BD465DF8047B7047380200203E
:1060F80080B582B000AF594B5B789BB208339BB236
:1061080019465648FEF7B2FE0346FB8000233B6063
:10611800FB88002B07D1FFF7CBFF034683F0010371
:10612800DBB2002B04D04D4B002283F8002192E013
:106138004A4B5B79CA2B61D0CA2B7BDCC82B02D0B7
:10614800C92B16D076E0454BD3F806303B603B6848
:10615800B3F5FA2F70DA00233B603B461946C82096
:10616800FFF73EFF3E4B00221A603E4B01221A60A9
:1061780062E03A4B9B791A46384BDB791B02134491
:10618800384A1268934228D1354B1B6803F10063E3
:1061980003F50033314A5278023AD10F0A445210BB
:1061A80092B231491846FEF7CDFE03463B603B6884
:1061B800032B43D12B4B1B6801332A4A1360274B0F
:1061C8005B781A46264B1B681344023B244A13602B
:1061D8002649C920FFF704FF30E0204B9B791A4677
:1061E8001E4BDB791B0213441A461E4B1B689A424E
:1061F80024D21E49C920FFF7F3FE1FE000233B60AD
:106208001B4B1B7883F00103DBB2002B18D0FEF781
:10621800F5FE03461A46164B1A70154B1B78002BD1
:1062280004D03B461946CA20FFF7DAFE3220FCF7B5
:10623800AFFB05E000BF04E000BF02E000BF00E0E4
:1062480000BF064B002283F800214FF48072002122
:10625800024800F06BF80837BD4680BD48040020AE
:106268008C05002090050020500400204E040020DA
:1062780094050020DFF834D00D480E490E4A00235B
:1062880002E0D458C4500433C4188C42F9D30B4AE2
:106298000B4C002301E013600432A242FBD3FFF74A
:1062A800C3FB00F011F8FEF781FF704700000220E1
:1062B80000000020400000208C65000840000020FD
:1062C8009C050020FEE7000070B50D4D0D4C641BC9
:1062D800A4100026A64209D10B4D0C4C00F02EF854
:1062E800641BA4100026A64205D170BD55F8043BD6
:1062F80098470136EEE755F8043B98470136F2E730
:1063080084650008846500088465000888650008BD
:106318000A44914200F1FF3300D1704710B511F8DB
:10632800014B03F8014F9142F9D110BD02440346D5
:10633800934200D1704703F8011BF9E7F8B500BF95
:10634800F8BC08BC9E467047F8B500BFF8BC08BC4E
:046358009E467047A6
:10635C00000610160006101600C1814001C08041D5
:10636C0001C0804100C1814001C0804100C1814019
:10637C0000C1814001C0804101C0804100C1814009
:10638C0000C1814001C0804100C1814001C08041F9
:10639C0001C0804100C1814001C0804100C18140E9
:1063AC0000C1814001C0804100C1814001C08041D9
:1063BC0001C0804100C1814000C1814001C08041C9
:1063CC0001C0804100C1814001C0804100C18140B9
:1063DC0000C1814001C0804101C0804100C18140A9
:1063EC0000C1814001C0804100C1814001C0804199
:1063FC0001C0804100C1814000C1814001C0804189
:10640C0001C0804100C1814001C0804100C1814078
:10641C0000C1814001C0804100C1814001C0804168
:10642C0001C0804100C1814001C0804100C1814058
:10643C0000C1814001C0804101C0804100C1814048
:10644C0000C1814001C0804100C1814001C0804138
:10645C0001C0804100C1814000C0C101C30302C220
:10646C00C60607C705C5C404CC0C0DCD0FCFCE0E88
:10647C000ACACB0BC90908C8D81819D91BDBDA1AF8
:10648C001EDEDF1FDD1D1CDC14D4D515D71716D668
:10649C00D21213D311D1D010F03031F133F3F232D8
:1064AC0036F6F737F53534F43CFCFD3DFF3F3EFE48
:1064BC00FA3A3BFB39F9F83828E8E929EB2B2AEAB8
:1064CC00EE2E2FEF2DEDEC2CE42425E527E7E62628
:1064DC0022E2E323E12120E0A06061A163A3A26298
:1064EC0066A6A767A56564A46CACAD6DAF6F6EAE08
:1064FC00AA6A6BAB69A9A86878B8B979BB7B7ABA78
:10650C00BE7E7FBF7DBDBC7CB47475B577B7B676E7
:10651C0072B2B373B17170B0509091519353529257
:10652C0096565797559594549C5C5D9D5F9F9E5EC7
:10653C005A9A9B5B99595898884849894B8B8A4A37
:10654C004E8E8F4F8D4D4C8C4484854587474686A7
:10655C008242438341818040000000000000000023
:10656C0001020304060708090000000001020304ED
:08657C007C9CFF7F0100000080
:04658400AD0100085D
:04658800890100087D
:10658C00100000000100000000000008004000089E
:10659C000080000800C0000800000108000002088C
:1065AC0000000408000006080000080800000A08A3
:1065BC0000000C0800000E08FF0000000024F4008E
:040000050800627D10
:00000001FF
